:100000000C942A000C9447000C9447000C94470071
:100010000C9449000C9447000C9447000C94470042
:100020000C9447000C9447000C9447000C94470034
:100030000C9447000C9447000C9447000C94470024
:100040000C9447000C9447000C9447000C94470014
:100050000C94470011241FBECFE5D8E0DEBFCDBF12
:1000600016E0A0E6B0E0EAE1FCE202C005900D92E5
:10007000AC36B107D9F717E0ACE6B6E001C01D9287
:10008000AA38B107E1F70E948B040C940B160C946C
:1000900000001F920F920FB60F9211248F939F931F
:1000A000AF93BF938091700690917106A0917206F4
:1000B000B09173060196A11DB11D809370069093B7
:1000C0007106A0937206B0937306BF91AF919F9192
:1000D0008F910F900FBE0F901F901895582F482F9B
:1000E0004F5F682F6F5E342F3F70E32FE695E695E4
:1000F000E695F0E0E856F94F808190E0232F2770D5
:1001000002C0959587952A95E2F780FD04C04F5F60
:10011000461749F7352F832F0895582F482F4F5FE3
:10012000682F6F5E342F3F70E32FE695E695E695D6
:10013000F0E0E550F94F808190E0232F277002C056
:10014000959587952A95E2F780FD04C04F5F461785
:1001500049F7352F832F089595B38F70907F892BA2
:1001600085BB08959BB38F70907F892B8BBB0895BF
:1001700081E080938006909198068091950698176B
:1001800031F49091990680919606981711F010928B
:10019000800680918006089581E080937A06909190
:1001A000FB0680914207981731F49091FC068091EC
:1001B0004307981711F010927A0680917A060895F5
:1001C00080E690E00E948206089584E492E00E9416
:1001D000820685E792E00E94820687E992E00E940B
:1001E000820681EC92E00E9482060895882321F025
:1001F0008FEE92E00E9482068091FC060E94D60655
:1002000080E20E9475068091FB060E94D60680E27D
:100210000E9475068AE00E947506809143070E943D
:10022000D60680E20E947506809142070E94D6069B
:100230000895882321F08EE093E00E948206809149
:1002400099060E94D60680E20E9475068091980663
:100250000E94D60680E20E9475068AE00E9475061A
:10026000809196060E94D60680E20E9475068091D3
:1002700095060E94D60680E20E94750608950F93A7
:100280001F931092FA0680E20E9475068BED96E0AD
:100290000E9482068AE00E94750690916C0699235E
:1002A00009F4A6C18091DB06823609F437C1833692
:1002B000A0F4873409F441C1883440F4843421F136
:1002C000853401F1813209F093C181C1883409F488
:1002D00095C1803509F08CC149C1873609F434C114
:1002E000883630F4843681F0853609F081C10AC041
:1002F000803709F430C1833709F442C1883609F0E8
:1003000077C17CC101E001C000E08091DC0682374A
:1003100031F0863721F0883611F0803739F4933088
:1003200040F01091DD0610531A3020F00E94E500D5
:100330005FC110E0943058F09091DE0690539A30EF
:1003400048F48AE0189F102D1124190F03C0933030
:1003500008F44EC182E693E00E948206002319F061
:1003600083E793E002C087E793E00E9482068091D2
:10037000DC06803709F498C0813720F4883609F00C
:10038000CAC068C0823721F0863709F0C4C031C0C6
:10039000E12FE695E695E695212F30E0002381F0E8
:1003A000F0E0E550F94F2770307081E090E002C036
:1003B000880F991F2A95E2F72081282B208316C0E9
:1003C000F0E02770307081E090E002C0880F991F44
:1003D0002A95E2F78095DF01A550B94F2C9128238B
:1003E0002C93EE5BF84F2081822380838CE793E08F
:1003F00088C0E12FE695E695E695212F30E00023B1
:1004000081F0F0E0E856F94F2770307081E090E01D
:1004100002C0880F991F2A95E2F72081282B20839C
:1004200016C0F0E02770307081E090E002C0880FC5
:10043000991F2A95E2F78095DF01A856B94F2C91B4
:1004400028232C93EB56F94F20818223808381E966
:1004500093E057C0212F30E0002379F023703070F3
:1004600081E090E002C0880F991F2A95E2F7209161
:100470009906282B2093990614C02370307081E0D0
:1004800090E002C0880F991F2A95E2F7809520918D
:10049000990628232093990620919606822380931B
:1004A000960683EA93E02DC0212F30E0002389F0E7
:1004B000237030702C5F3F4F81E090E002C0880FC6
:1004C000991F2A95E2F720919906282B20939906E7
:1004D00016C0237030702C5F3F4F81E090E002C067
:1004E000880F991F2A95E2F7809520919906282375
:1004F000209399062091960682238093960686EB98
:1005000093E00E948206812F62E00E94E5068AE065
:100510000E9475066DC089EC93E068C088E094E0A5
:100520000E94820681E0809397068091DC068033EA
:1005300009F061C01092970657C0109211051092F1
:1005400042071092430754C010921305109295066B
:10055000109296064DC081E0809381068091DC0662
:10056000803309F045C01092810642C081E080933B
:100570007B068091DC068033D9F510927B0638C06B
:1005800081E00E9419018AE00E94750681E00E94C4
:10059000F6008AE00E9475068DE194E00E948206D2
:1005A0006091700670917106809172069091730649
:1005B0000E94111320E030E04AE754E40E945311F6
:1005C00041E027E00E94B30683E294E00FC08AE294
:1005D00094E00E94820681E0809382068091DC068E
:1005E000803349F41092820684E194E00E948206EE
:1005F000EBEDF6E006C089E194E0F8CF80E690E00C
:10060000F5CF119286E0EB3FF807D9F71F910F91D4
:100610000895BF92CF92DF92EF92FF920F931F93B4
:10062000CF93DF93B62E8823C1F087E394E00E9436
:10063000820610E086E794E00E948206812F62E045
:100640000E94E50689E794E00E9482061F5F103150
:1006500089F78DE794E00E9482068CE70E94750678
:100660008BE9C82E86E0D82EC0E0D0E0CE0186957A
:1006700086958695E82FF0E0E550F94F808190E06F
:100680009E012770307002C0959587952A95E2F7F4
:1006900080FF54C060910D0570910E0580910F058B
:1006A0009091100520E030E040E854E40E94591099
:1006B0007B018C01F60160817181828193810E94AE
:1006C00011139B01AC01C801B7010E94591020E031
:1006D00030E040E053E30E9459107B018C0120E0A0
:1006E00030E04AE754E40E942F1288231CF480E291
:1006F0000E947506C801B70120E030E048EC52E4E2
:100700000E942F1288231CF480E20E947506C80103
:10071000B70120E030E040E251E40E942F1288232C
:100720001CF480E20E947506C801B70141E025E093
:100730000E94B3068CE70E94750604C080E894E02E
:100740000E948206219684E090E0C80ED91EC03136
:10075000D10509F08BCFBB2019F08AE00E94750605
:10076000DF91CF911F910F91FF90EF90DF90CF908D
:10077000BF900895FF920F931F93CF93DF93F62EB0
:10078000882309F478C088E894E00E94820610E08B
:1007900086EB94E00E948206812F61E00E94E506CC
:1007A00089E794E00E9482061F5F183089F78AEB80
:1007B00094E00E94820680E061E00E94E50689E7FD
:1007C00094E00E9482068AEB94E00E94820681E017
:1007D00061E00E94E50689E794E00E9482068AEBC8
:1007E00094E00E94820682E061E00E94E50689E7CB
:1007F00094E00E9482068AEB94E00E94820683E0E5
:1008000061E00E94E50689E794E00E9482068EEB93
:1008100094E00E94820680E061E00E94E50689E79C
:1008200094E00E9482068EEB94E00E94820681E0B2
:1008300061E00E94E50689E794E00E9482068EEB63
:1008400094E00E94820682E061E00E94E50689E76A
:1008500094E00E9482068EEB94E00E94820683E080
:1008600061E00E94E50689E794E00E9482068DE738
:1008700094E00E94820602E017E0C0E0D0E08CE73E
:100880000E947506CE01869586958695E82FF0E044
:10089000E856F94F808190E09E012770307002C0C9
:1008A000959587952A95E2F780FF1DC0F801608134
:1008B00071818281938122E0660F771F881F991FC3
:1008C0002A95D1F76E5F7F4F8F4F9F4F2091120572
:1008D00030E040E050E00E94B215CA01B90146E0A4
:1008E0000E94C20604C082EC94E00E948206219617
:1008F0000C5F1F4FC031D10511F68CE70E947506C1
:10090000FF2019F08AE00E947506DF91CF911F91B8
:100910000F91FF900895CF92DF92EF92FF920F9385
:100920001F93CF93DF930E94EA060E9469060E94FC
:1009300051070E94CE080E944B0988E085BD85B50D
:10094000836085BD8CE783BD89B7806889BF789453
:10095000C2989FEF109242071092FC069093FB06FC
:10096000109243071092950683E380939906909323
:1009700098061092960684E195E00E94820680E631
:1009800090E00E94820681E00E9419018AE00E94A4
:10099000750681E00E94F6008AE00E9475068DE1EE
:1009A00094E00E94820660917006709171068091B9
:1009B0007206909173060E94111320E030E04AE71E
:1009C00054E40E94531141E027E00E94B30683E201
:1009D00094E00E94820611E000E181E0E82EF12C13
:1009E000B0E2CB2EBEE4DB2E0E94B800882379F162
:1009F00080918106882309F189EC94E00E948206A7
:100A000060917006709171068091720690917306E4
:100A10000E94111320E030E04AE754E40E94531191
:100A200041E024E00E94B30680E061E00E94BA0346
:100A300010929506109296060AC08091130588239D
:100A400031F41093130581E061E00E94BA030E9423
:100A5000CC00882379F180917B06882309F18CEC06
:100A600094E00E94820660917006709171068091F8
:100A70007206909173060E94111320E030E04AE75D
:100A800054E40E94531141E024E00E94B30680E048
:100A900061E00E94090310924207109243070AC0C6
:100AA00080911105882331F41093110581E061E0F4
:100AB0000E94090380919706882319F08BB3802741
:100AC0008BBB90916D06992381F05D9B0EC0809148
:100AD000FD068CB9EDEFF6E08181819347E0E230CD
:100AE000F407D1F7915090936D065F9B1CC09CB1A9
:100AF00090939A0680916C06803278F4E82FF0E0AB
:100B0000E552F94F90838F5F80936C0681509A3045
:100B100051F480936C06108204C08FEC94E00E9424
:100B2000820610936F065B9B07C088EF94E00E94DB
:100B300082068CB180939A0680916F06882369F0B3
:100B40000E943F0110926F06EBEDF6E0119256E025
:100B5000EB3FF507D9F710926C06349B60C080918B
:100B60008006882309F05BC084B195B1D92FC0E01D
:100B7000AE01480F511D50937F0640937E06609151
:100B80007C068091120530917D06681771F5E32F80
:100B9000E695E695E695F0E0EB56F94F832F8770E2
:100BA000A70102C0440F551F8A95E2F72081242B2C
:100BB0002083832F0E946E0080937D06E82FF0E053
:100BC000EE0FFF1FEE0FFF1FEE5FF84F1082118236
:100BD0001282138295B38F70907F982B95BB1092E1
:100BE0007C06C6010197F1F71AC0E32FF0E0EE0F83
:100BF000FF1FEE0FFF1FEE5FF84FCA01A0E0B0E04D
:100C00002081318142815381820F931FA41FB51F20
:100C100080839183A283B3836F5F60937C06829904
:100C2000E3CE80917A06882309F0DECE0E94780810
:100C30006093760670937706809378069093790692
:100C400020917406309182062230B9F5E091750644
:100C5000F0E0EE0FFF1FEE0FFF1FE556F94F608328
:100C600071838283938310927406332341F00E9430
:100C7000B8068AE00E9475068AE00E947506809197
:100C80007506E82FE695E695E695F0E0EE5BF84F01
:100C9000282F2770A70102C0440F551F2A95E2F79D
:100CA0009081942B90830E948D00809375069BB356
:100CB0008F70907F982B9BBB97CE2F5F20937406ED
:100CC000332309F491CE0E94B8068AE00E9475068B
:100CD0008BCE10BC83E389B91BB81AB8549A889894
:100CE000539A899A86E880BD08955D9BFECF8CB9A2
:100CF00008955D9BFECF8DE08CB95D9BFECF8AE0B1
:100D00008CB90895FC0104C05D9BFECF31968CB96F
:100D100080818823C9F70895FC0104C05D9BFECF44
:100D200031968CB980818823C9F70895FC0104C0ED
:100D30005D9BFECF31968CB980818823C9F75D9B7E
:100D4000FECF8DE08CB95D9BFECF8AE08CB9089513
:100D50000E9482065D9BFECF8DE08CB95D9BFECF2D
:100D60008AE08CB908950E941B0A0E9482060895A9
:100D70000E94B4090E94820608950E94120B0E94EC
:100D8000820608950E942F0C0E94820608950E94F8
:100D90008E090E94820608950E944B0D0E948206D1
:100DA00008950E94AE0D0E94820608950E94720965
:100DB0000E94820608950E945C090E94820608959E
:100DC0000E940A0E0E94820608950E94480E0E9408
:100DD0008206089584B78093440714BE8898899A40
:100DE000D598D698D498D598D698D798D49AD79895
:100DF0008AB38F608ABB84B38F6084BBBB9ABC9A72
:100E0000C39AC49ABD9ABF9ABE98C59AC79A8A983F
:100E1000B99AB89808952FB78D5FF894A89591B5B1
:100E2000986191BD81BD2FBF08951DB8809159076C
:100E300080FF02C06D9A01C06D988DB18091460708
:100E400080FF02C06B9A01C06B988DB180915707EB
:100E500080FF02C06A9A01C06A988DB180915807DC
:100E6000833091F0843028F4813051F0823050F496
:100E700010C0853089F0853048F0863051F407C0C5
:100E8000699A0AC0699A03C0689A06C0689A709AFB
:100E900004C08DB183608DB970988DB180658DB9B6
:100EA0000895109258071092590781E080934607E1
:100EB000809357070E9415070895873008F086E051
:100EC000809358070E9415070895811181E080934F
:100ED00059070E9415070895811181E08093460704
:100EE0000E9415070895811181E0809357070E94A1
:100EF000150708956C9B6C9A8FB9779BFECF8FB1C5
:100F00000895AF92BF92CF92DF92EF92FF920F932C
:100F10001F93CF93DF93C82ED62EEE24FF24862F67
:100F200090E023E8A22E26E0B22EA80EB91EEC0116
:100F3000C05BDA4F01E010E07BC0F50180818823BF
:100F4000C1F0DD2059F428B38881A80102C0440F04
:100F5000551F8A95E2F7242B28BB26C022B388812F
:100F6000F80102C0EE0FFF1F8A95E2F72E2B22BB7D
:100F70001BC0DD2069F428B38881A80102C0440F9A
:100F8000551F8A95E2F7CA018095822388BB0CC061
:100F900022B38881F80102C0EE0FFF1F8A95E2F7A5
:100FA000CF018095822382BBF701E95BF84F8081F6
:100FB0000E947A07F701E65AF84F8083F501808195
:100FC0008823E1F0DD2069F428B38881A80102C0FC
:100FD000440F551F8A95E2F7CA018095822388BB8A
:100FE00024C022B38881F80102C0EE0FFF1F8A954A
:100FF000E2F7CF018095822382BB17C0DD2059F430
:1010000028B38881A80102C0440F551F8A95E2F7D2
:10101000242B28BB0AC022B38881F80102C0EE0F3E
:10102000FF1F8A95E2F72E2B22BB0894E11CF11CCE
:10103000EC1408F482CFDF91CF911F910F91FF90B4
:10104000EF90DF90CF90BF90AF900895FF920F93F5
:101050001F93CF93DF93F82E042F442379F488B3A2
:101060009091500521E030E002C0220F331F9A9585
:10107000E2F7822788BBEB0110E014C022B3E42F13
:10108000F0E0E05BFA4F308181E090E002C0880F31
:10109000991F3A95E2F7282722BBEDCF89910E944C
:1010A0007A071F5F1F15D0F3002369F488B390916E
:1010B000500521E030E002C0220F331F9A95E2F77D
:1010C000822788BB0FC022B3E02FF0E0E05BFA4F2D
:1010D000308181E090E002C0880F991F3A95E2F7D5
:1010E000282722BBDF91CF911F910F91FF90089588
:1010F000EF92FF920F931F93C49885E40E947A07A2
:10110000C49A85E88A95F1F7C49880E00E947A072E
:10111000E82EFF2400E010E0102F0F2DFE2CEE240F
:1011200080E00E947A0790E0A0E0B0E0E82AF92A87
:101130000A2B1B2B102F0F2DFE2CEE2480E00E947B
:101140007A07C49A282F30E040E050E02E293F294A
:10115000402B512BB901CA011F910F91FF90EF90C5
:101160000895C49881E00E947A07C49AC49881E0E7
:101170000E947A07C49A08951F93182FC49881E09B
:101180000E947A07C49AC498112311F082E001C02A
:1011900083E00E947A07C49A1F9108951F93C19813
:1011A000C19AC49884E40E947A07C49A15E8812FF2
:1011B0008A95F1F7C49880E00E947A07C49A812F3B
:1011C0008A95F1F7C49887E00E947A07C49A812F24
:1011D0008A95F1F7C49883E00E947A07C49A812F18
:1011E0008A95F1F7C49880E00E947A07C49A812F0B
:1011F0008A95F1F7C49884E00E947A07C49A812FF7
:101200008A95F1F7C49882E50E947A07C49A812FE3
:101210008A95F1F7C49883E00E947A07C49A812FD7
:101220008A95F1F7C49881E30E947A07C49A812FC6
:101230008A95F1F7C49882E00E947A07C49A812FB8
:101240008A95F1F7C4988EE80E947A07C49A812F94
:101250008A95F1F7C49881E00E947A07C49A812F99
:101260008A95F1F7C49883E00E947A07C49A812F87
:101270008A95F1F7C49884E40E947A07C49A812F72
:101280008A95F1F7C49880E00E947A07C49A1A956B
:10129000F1F71F91089586B1866086B93098359A26
:1012A00080B78F7180BF379A3E983F983D9887B13D
:1012B000876087B9369A0895982F92959F70A2E516
:1012C000B5E0FD01E90FF11D908190936A078F70E1
:1012D000A80FB11D8C9180936B0710926C078AE662
:1012E00097E00895EAE6F7E027E0482F50E060E352
:1012F00031E3CA01022E02C0959587950A94E2F760
:10130000DF01119680FF02C0308301C06083FD01C0
:10131000215078F71C928AE697E00895292F2295AC
:101320002F70A2E5B5E0FD01E20FF11D20812093B1
:101330006A079F70FD01E90FF11D908190936B0783
:10134000982F92959F70FD01E90FF11D9081909368
:101350006C078F70A80FB11D8C9180936D07109250
:101360006E078AE697E00895292F22952F70A2E54F
:10137000B5E0FD01E20FF11D208120936A079F7007
:10138000FD01E90FF11D908190936B07982F9295C5
:101390009F70FD01E90FF11D908190936C078F7094
:1013A000FD01E80FF11D808180936D07872F8295E5
:1013B0008F70FD01E80FF11D808180936E077F70B3
:1013C000FD01E70FF11D808180936F07862F8295C5
:1013D0008F70FD01E80FF11D8081809370076F70A1
:1013E000A60FB11D8C9180937107109272078AE647
:1013F00097E00895CF93DF93EC01FC01019000206A
:10140000E9F73197E81BAAE7B7E080E202C08D93C5
:101410006150E617E0F3CD018E0F911DFC0102C073
:1014200089918D93AE17BF07D9F71C928AE797E091
:10143000DF91CF9108952F923F924F925F926F92DA
:101440007F928F929F92AF92BF92CF92DF92EF9254
:10145000FF920F931F93DF93CF930F92CDB7DEB719
:101460003B014C012983242E85E0841710F435E0DC
:10147000232EC401B30120E030E040E050E00E94A0
:101480002F1287FD05C02AE6422E27E0522E0BC000
:101490008DE280936A0797FA909497F890949BE670
:1014A000492E97E0592EC401B3010E94830E5B01BF
:1014B0006C01611571058105910521F480E3D2016C
:1014C0008D932D0186017501332423C0C801B70116
:1014D0002AE030E040E050E00E94B215E32DF0E059
:1014E000EB57F94F6083E61AF10801091109E1147D
:1014F000F1040105110561F0C801B7012AE030E0EF
:1015000040E050E00E94B215C901DA017C018D0172
:101510003394E114F10401051105C1F6C601B501CA
:101520000E9411139B01AC01C401B3010E94FB0F87
:101530007B018C018DE8A82E86E0B82E6501822CF7
:1015400099243501680C791C22C0C801B70120E03C
:1015500030E040E251E40E9459107B018C010E946E
:10156000830EF6016083662379F070E0882777FDAB
:101570008095982F0E945F129B01AC01C801B701B2
:101580000E94FB0F7B018C010894C11CD11CC61466
:10159000D704D9F6932D9150A92FBB27A7FDB0955D
:1015A000AB57B94F07C08C91805DF2018083290150
:1015B0009150119792012F5F3F4F97FFF4CF8EE22A
:1015C000D2018C93F20105C0D5018D915D01805D42
:1015D00080833196AC14BD04B9F7280D391DF9018B
:1015E0001082F981FF2319F42AE637E006C08AE663
:1015F00097E069810E94FA099C01C9010F90CF917F
:10160000DF911F910F91FF90EF90DF90CF90BF90EF
:10161000AF909F908F907F906F905F904F903F9092
:101620002F900895BF92CF92DF92EF92FF920F9387
:101630001F93CF93DF938B019C01B42E97FF0DC0B6
:101640008DE280936A07CC24DD247601C01AD10A8A
:10165000E20AF30ACBE6D7E004C06B017C01CAE6DC
:10166000D7E080E0C8168AECD8068AE9E8068BE362
:10167000F80658F0C701B60120E03AEC4AE95BE30E
:101680000E94B215205D299309C080E0C81681EE42
:10169000D80685EFE80685E0F80688F0C701B601B0
:1016A00020E03AEC4AE95BE30E94B21520E031EE1B
:1016B00045EF55E00E94B215205D299309C080E8EE
:1016C000C81686E9D80688E9E80680E0F80688F0BA
:1016D000C701B60120E031EE45EF55E00E94B2159A
:1016E00020E836E948E950E00E94B215205D2993D0
:1016F00009C080E4C81682E4D8068FE0E80680E0DE
:10170000F80688F0C701B60120E836E948E950E05C
:101710000E94B21520E432E44FE050E00E94B2157E
:10172000205D299309C080EAC81686E8D80681E0C2
:10173000E80680E0F80688F0C701B60120E432E44C
:101740004FE050E00E94B21520EA36E841E050E058
:101750000E94B215205D299309C080E1C81687E276
:10176000D80680E0E80680E0F80688F0C701B601F8
:1017700020EA36E841E050E00E94B21520E137E26D
:1017800040E050E00E94B215205D299309C088EE28
:10179000C81683E0D80680E0E80680E0F80688F006
:1017A000C701B60120E137E240E050E00E94B215E7
:1017B00028EE33E040E050E00E94B215205D29930E
:1017C00006C084E6C816D104E104F10488F0C7011C
:1017D000B60128EE33E040E050E00E94B21524E666
:1017E00030E040E050E00E94B215205D299306C031
:1017F0008AE0C816D104E104F10480F0C701B60103
:1018000024E630E040E050E00E94B2152AE030E0EB
:1018100040E050E00E94B215205D2993C701B60157
:101820002AE030E040E050E00E94B215605D68833D
:101830001982BB2019F42AE637E006C08AE697E051
:101840006B2D0E94FA099C01C901DF91CF911F9174
:101850000F91FF90EF90DF90CF90BF900895DF92AF
:10186000EF92FF920F931F93CF93DF937B018C0135
:10187000D42E80E0E8168AECF8068AE908078BE3A4
:10188000180770F0C801B70120E03AEC4AE95BE3C1
:101890000E94B215205D20936A07CBE6D7E00BC00B
:1018A00080E0E81681EEF80685EF080785E0180766
:1018B00098F0CAE6D7E0C801B70120E03AEC4AE95F
:1018C0005BE30E94B21520E031EE45EF55E00E9447
:1018D000B215205D29930BC080E8E81686E9F8066A
:1018E00088E9080780E0180798F0CAE6D7E0C80141
:1018F000B70120E031EE45EF55E00E94B21520E837
:1019000036E948E950E00E94B215205D29930BC0EA
:1019100080E4E81682E4F8068FE0080780E0180704
:1019200098F0CAE6D7E0C801B70120E836E948E9EF
:1019300050E00E94B21520E432E44FE050E00E94F3
:10194000B215205D29930BC080EAE81686E8F806F8
:1019500081E0080780E0180798F0CAE6D7E0C801E0
:10196000B70120E432E44FE050E00E94B21520EAD3
:1019700036E841E050E00E94B215205D29930BC08B
:1019800080E1E81687E2F80680E0080780E01807A3
:1019900098F0CAE6D7E0C801B70120EA36E841E08E
:1019A00050E00E94B21520E137E240E050E00E9492
:1019B000B215205D29930BC088EEE81683E0F80687
:1019C00080E0080780E0180798F0CAE6D7E0C80171
:1019D000B70120E137E240E050E00E94B21528EE66
:1019E00033E040E050E00E94B215205D299308C02A
:1019F00084E6E816F1040105110598F0CAE6D7E07F
:101A0000C801B70128EE33E040E050E00E94B21573
:101A100024E630E040E050E00E94B215205D2993BA
:101A20000BC08AE0E816F1040105110518F4CAE6B6
:101A3000D7E012C0CAE6D7E0C801B70124E630E01B
:101A400040E050E00E94B2152AE030E040E050E073
:101A50000E94B215205D2993C801B7012AE030E049
:101A600040E050E00E94B215605D68831982DD207D
:101A700019F42AE637E006C08AE697E06D2D0E9449
:101A8000FA099C01C901DF91CF911F910F91FF903D
:101A9000EF90DF900895CF93DF939C01462F97FF3F
:101AA0000AC08DE280936A07EE27FF27E21BF30B43
:101AB000CBE6D7E003C0FC01CAE6D7E087E2E0311D
:101AC000F80740F0CF0160E177E20E948B15605D7E
:101AD000699304C083E0E83EF80760F0CF0160E15D
:101AE00077E20E948B1568EE73E00E948B15605DB3
:101AF000699303C0E436F10560F0CF0168EE73E04E
:101B00000E948B1564E670E00E948B15605D6993FE
:101B100003C0EA30F10558F0CF0164E670E00E949E
:101B20008B156AE070E00E948B15605D6993CF01B0
:101B30006AE070E00E948B15805D888319824423DF
:101B400019F42AE637E006C08AE697E0642F0E947F
:101B5000FA099C01C901DF91CF9108959C01462F9C
:101B600087E22031380758F0C90160E177E20E942E
:101B70008B15605D60936A07EBE6F7E006C083E0D3
:101B8000283E380770F0EAE6F7E0C90160E177E245
:101B90000E948B1568EE73E00E948B15605D619367
:101BA00005C02436310570F0EAE6F7E0C90168EEB9
:101BB00073E00E948B1564E670E00E948B15605DF7
:101BC000619308C02A30310518F4EAE6F7E00DC049
:101BD000EAE6F7E0C90164E670E00E948B156AE06E
:101BE00070E00E948B15605D6193C9016AE070E04E
:101BF0000E948B15805D80831182442319F42AE6AC
:101C000037E006C08AE697E0642F0E94FA099C013B
:101C1000C9010895982F362F87FF08C08DE2809361
:101C20006A07292F2195EBE6F7E003C0282FEAE6A3
:101C3000F7E0243668F0822F90E068EE73E00E94AF
:101C40009F1564E670E00E949F15605D619302C07D
:101C50002A3050F0822F64E60E947F15892F6AE0B7
:101C60000E947F15805D8193822F6AE00E947F151C
:101C7000905D90831182332319F42AE637E006C081
:101C80008AE697E0632F0E94FA099C01C901089532
:101C90001F93482F162F843678F090E068EE73E09B
:101CA0000E949F1564E670E00E949F15605D60933E
:101CB0006A072BE637E007C08A3018F4EAE6F7E057
:101CC0000DC02AE637E0842F64E60E947F15892F35
:101CD0006AE00E947F15805DF9018193842F6AE09C
:101CE0000E947F15905D90831182112319F42AE6DA
:101CF00037E006C08AE697E0612F0E94FA099C014E
:101D0000C9011F910895EF92FF920F931F937B01DA
:101D10008C0120E030E040E05FE40E94FF11882366
:101D20008CF0C801B70120E030E040E05FE40E94A1
:101D3000FB0F0E94BD129B01AC012050304040407F
:101D4000504806C0C801B7010E94BD129B01AC01FA
:101D5000B901CA011F910F91FF90EF900895A0E083
:101D6000B0E0E5EBFEE00C94D415DC012B01FA01A8
:101D70009C91923008F439C1EB018881823008F4DB
:101D800033C1943069F4843009F02FC111969C91CD
:101D900011978981981709F428C1A3E6B5E025C1F8
:101DA000843009F421C18230A9F4923009F01DC1B8
:101DB0009A01AD0188E0EA010990AE01E9010992BA
:101DC0009E018150C1F7E201898111969C9189237E
:101DD000818308C1923009F407C112962D903C907E
:101DE0001397EB018A819B811496AD90BD90CD90A5
:101DF000DC901797EC80FD800E811F819101281BDC
:101E0000390BB90137FF04C066277727621B730BB4
:101E1000603271050CF061C0121613066CF53701C3
:101E20004801062E04C096948794779467940A9488
:101E3000D2F721E030E040E050E004C0220F331F31
:101E4000441F551F6A95D2F7215030404040504002
:101E50002E213F21402351232115310541055105F4
:101E600021F021E030E040E050E079018A01E628ED
:101E7000F728082919293CC0232BD1F1260E371E3B
:101E800035014601062E04C0969487947794679492
:101E90000A94D2F721E030E040E050E004C0220F85
:101EA000331F441F551F6A95D2F7215030404040E0
:101EB00050402A213B214C215D212115310541054E
:101EC000510521F021E030E040E050E059016A0185
:101ED000A628B728C828D9280BC0821593052CF04E
:101EE0001C01AA24BB24650103C0EE24FF24870142
:101EF00011969C91D20111968C91981709F445C0C6
:101F0000992339F0A80197012A193B094C095D0969
:101F100006C0A60195012E193F09400B510B57FD34
:101F200008C01182338222822483358346835783FB
:101F30001DC081E081833382228288279927DC01BA
:101F4000821B930BA40BB50B84839583A683B78365
:101F50000DC0220F331F441F551F24833583468332
:101F60005783828193810197938382832481358172
:101F700046815781DA01C9010197A109B1098F5F33
:101F80009F4FAF4FBF4328F30BC091833382228210
:101F9000EA0CFB1C0C1D1D1DE482F58206831783D1
:101FA00083E08083248135814681578157FF1AC0A1
:101FB000C901AA2797FDA095BA2F81709070A070D3
:101FC000B0705695479537952795822B932BA42B68
:101FD000B52B84839583A683B783828193810196F1
:101FE00093838283DF0101C0D201CD01CDB7DEB77B
:101FF000E2E10C94F015A0E2B0E0E1E0F0E10C9435
:10200000E01569837A838B839C832D833E834F8382
:102010005887E9E0EE2EF12CEC0EFD1ECE01019664
:10202000B7010E94AE148E010F5E1F4FCE010596C0
:10203000B8010E94AE148A8991E089278A8BC70172
:10204000B801AE01475E5F4F0E94AF0E0E94D913E8
:10205000A096E6E00C94FC15A0E2B0E0E2E3F0E12B
:102060000C94E01569837A838B839C832D833E8354
:102070004F835887F9E0EF2EF12CEC0EFD1ECE01B8
:102080000196B7010E94AE148E010F5E1F4FCE0164
:102090000596B8010E94AE14C701B801AE01475EB3
:1020A0005F4F0E94AF0E0E94D913A096E6E00C94F9
:1020B000FC15A0E2B0E0EFE5F0E10C94D4156983E3
:1020C0007A838B839C832D833E834F835887CE01F5
:1020D0000196BE01675F7F4F0E94AE14CE01059648
:1020E000BE016F5E7F4F0E94AE149985923088F0DA
:1020F00089898230C8F0943019F4823051F404C0D8
:10210000843029F4923081F483E695E0C6C09230A1
:1021100049F420E09A858A89981321E02A87CE0124
:102120000996BBC0823049F420E09A858A899813C9
:1021300021E02A8BCE014196B0C02D843E844F848D
:1021400058886D887E888F88988CEE24FF248701BC
:10215000AA24BB24650140E050E060E070E0E0E0CC
:10216000F0E0C10181709070892BE9F0E60CF71C5A
:10217000081D191D9A01AB012A0D3B1D4C1D5D1D4B
:1021800080E090E0A0E0B0E0E614F704080519054F
:1021900020F481E090E0A0E0B0E0BA01A901480F8E
:1021A000591F6A1F7B1FAA0CBB1CCC1CDD1C97FE91
:1021B00008C081E090E0A0E0B0E0A82AB92ACA2ACD
:1021C000DB2A3196E032F10549F0660C771C881C59
:1021D000991C5694479437942794C3CFFA85EA897B
:1021E0002B893C898B859C85280F391F2E5F3F4F9B
:1021F00017C0CA0181709070892B61F01695079500
:10220000F794E79480E090E0A0E0B0E8E82AF92AAB
:102210000A2B1B2B76956795579547952F5F3F4F58
:1022200077FDE7CF0CC0440F551F661F771F17FDC2
:102230004160EE0CFF1C001F111F21503040403048
:1022400090E0590790E0690790E4790760F32B8FDD
:102250003C8FDB01CA018F779070A070B070803422
:102260009105A105B10561F447FD0AC0E114F1042F
:102270000105110529F0405C5F4F6F4F7F4F40789B
:102280001A8EFE1711F081E08A8F4D8F5E8F6F8F4F
:1022900078A383E0898FCE0149960E94D913A09636
:1022A000E2E10C94F015A8E1B0E0E9E5F1E10C946D
:1022B000DC1569837A838B839C832D833E834F83D4
:1022C0005887B9E0EB2EF12CEC0EFD1ECE010196E5
:1022D000B7010E94AE148E010F5E1F4FCE0105960E
:1022E000B8010E94AE142985223008F47EC03989D5
:1022F000323010F4B8017CC08A859A8989278A8790
:10230000243011F0223031F4231709F06EC063E657
:1023100075E06EC0343039F41D861E861F86188A1B
:102320001C861B8604C0323021F484E08987B70103
:102330005FC02B853C858B899C89281B390B3C878A
:102340002B87ED84FE840F851889AD88BE88CF88E1
:10235000D88CEA14FB040C051D0540F4EE0CFF1CA0
:10236000001F111F215030403C872B8720E030E0B8
:1023700040E050E080E090E0A0E0B0E460E070E099
:10238000EA14FB040C051D0540F0282B392B4A2BC1
:102390005B2BEA18FB080C091D09B695A7959795C4
:1023A0008795EE0CFF1C001F111F6F5F7F4F6F3171
:1023B000710531F7DA01C9018F779070A070B070A4
:1023C00080349105A105B10561F427FD0AC0E1142F
:1023D000F1040105110529F0205C3F4F4F4F5F4F7D
:1023E00020782D873E874F87588BBE01675F7F4FD0
:1023F000CB010E94D9136896EAE00C94F815A8E185
:10240000B0E0E5E0F2E10C94E01569837A838B8318
:102410009C832D833E834F83588789E0E82EF12CDF
:10242000EC0EFD1ECE010196B7010E94AE148E0186
:102430000F5E1F4FCE010596B8010E94AE1489852C
:10244000823040F08989823028F0C701B8010E94AB
:10245000261501C08FEF6896E6E00C94FC15A8E104
:10246000B0E0E5E3F2E10C94E01569837A838B83B5
:102470009C832D833E834F83588789E0E82EF12C7F
:10248000EC0EFD1ECE010196B7010E94AE148E0126
:102490000F5E1F4FCE010596B8010E94AE148985CC
:1024A000823040F08989823028F0C701B8010E944B
:1024B000261501C081E06896E6E00C94FC15A8E0C2
:1024C000B0E0E5E6F2E10C94DD159B01AC0183E0A0
:1024D0008983DA01C9018827B7FD83959927AA273F
:1024E000BB27B82E211531054105510519F482E0AD
:1024F00089833AC08823A9F0203080E0380780E043
:10250000480780E8580729F460E070E080E09FEC1D
:1025100030C0EE24FF248701E21AF30A040B150BE6
:1025200002C079018A018EE1C82ED12CDC82CB82D7
:10253000ED82FE820F831887C801B7010E948A13BB
:1025400001971816190684F4082E04C0EE0CFF1C1F
:10255000001F111F0A94D2F7ED82FE820F831887A5
:10256000C81AD90ADC82CB82BA82CE0101960E94B7
:10257000D9132896E9E00C94F915ACE0B0E0E3EC4F
:10258000F2E10C94E41569837A838B839C83CE01FA
:102590000196BE016B5F7F4F0E94AE148D81823029
:1025A00061F1823050F1843021F48E81882351F121
:1025B0002EC02F81388537FD20C06E812F31310527
:1025C0001CF06623F9F023C08EE190E0821B930B90
:1025D00029853A854B855C8504C056954795379586
:1025E00027958A95D2F76623B1F05095409530959E
:1025F00021953F4F4F4F5F4F0EC020E030E040E04D
:1026000050E009C02FEF3FEF4FEF5FE704C020E03D
:1026100030E040E050E8B901CA012C96E2E00C94A9
:102620000016A8E0B0E0E7E1F3E10C94DC157B01D3
:102630008C01611571058105910519F482E089838A
:1026400060C083E089838EE1C82ED12CDC82CB82EE
:10265000ED82FE820F831887C801B7010E948A139A
:10266000FC013197F7FF3BC0222733272E1B3F0B7E
:1026700057016801022E04C0D694C794B794A7945A
:102680000A94D2F740E050E060E070E081E090E032
:10269000A0E0B0E004C0880F991FAA1FBB1F2A95B5
:1026A000D2F70197A109B1098E219F21A023B1235F
:1026B0000097A105B10521F041E050E060E070E035
:1026C0004A295B296C297D294D835E836F83788736
:1026D0008EE190E08E1B9F0B9C838B8312C0309702
:1026E00081F00E2E04C0EE0CFF1C001F111F0A9477
:1026F000D2F7ED82FE820F831887CE1ADF0ADC82C2
:10270000CB821A82CE0101960E94D9132896EAE064
:102710000C94F815EF92FF920F931F937B018C019D
:1027200080E0E81680E0F80681E0080780E01807FE
:1027300088F48FEFE816F1040105110531F028F057
:1027400088E090E0A0E0B0E017C080E090E0A0E07A
:10275000B0E012C080E0E81680E0F80680E00807EC
:1027600081E0180728F088E190E0A0E0B0E004C024
:1027700080E190E0A0E0B0E020E230E040E050E016
:10278000281B390B4A0B5B0B04C016950795F79471
:10279000E7948A95D2F7F701E559FA4F8081281B13
:1027A000310941095109C9011F910F91FF90EF9023
:1027B0000895DF92EF92FF920F931F93FC01E48044
:1027C000F58006811781D1808081823048F480E0D5
:1027D00090E0A0E1B0E0E82AF92A0A2B1B2BA5C063
:1027E000843009F49FC0823021F4EE24FF24870155
:1027F00005C0E114F1040105110519F4E0E0F0E071
:1028000096C0628173819FEF623879070CF05BC0DC
:1028100022E83FEF261B370B2A3131052CF020E050
:1028200030E040E050E02AC0B801A701022E04C009
:1028300076956795579547950A94D2F781E090E091
:10284000A0E0B0E004C0880F991FAA1FBB1F2A9503
:10285000D2F70197A109B1098E219F21A023B123AD
:102860000097A105B10521F081E090E0A0E0B0E083
:102870009A01AB01282B392B4A2B5B2BDA01C901BA
:102880008F779070A070B07080349105A105B1056C
:1028900039F427FF09C0205C3F4F4F4F5F4F04C002
:1028A000215C3F4F4F4F5F4FE0E0F0E02030A0E071
:1028B0003A07A0E04A07A0E45A0710F0E1E0F0E090
:1028C00079018A0127C06038710564F5FB01E15880
:1028D000FF4FD801C7018F779070A070B07080341F
:1028E0009105A105B10539F4E7FE0DC080E490E043
:1028F000A0E0B0E004C08FE390E0A0E0B0E0E80E1C
:10290000F91E0A1F1B1F17FF05C016950795F794A0
:10291000E794319687E016950795F794E7948A95A2
:10292000D1F705C0EE24FF248701EFEFF0E06E2F12
:10293000679566276795902F9F77D794DD24D79466
:102940008E2F8695492F462B582F5D29B701CA0136
:102950001F910F91FF90EF90DF900895FC01DB0134
:10296000408151812281622F6F7770E0221F2227E0
:10297000221F9381892F880F822B282F30E0991FE7
:102980009927991F11969C93119721153105A9F547
:10299000411551056105710511F482E037C082E8E7
:1029A0009FEF13969C938E9312979A01AB0167E069
:1029B000220F331F441F551F6A95D1F783E08C9374
:1029C0000DC0220F331F441F551F12968D919C91ED
:1029D0001397019713969C938E931297203080E063
:1029E000380780E0480780E4580758F314962D9381
:1029F0003D934D935C93179708952F3F310579F4DC
:102A0000411551056105710519F484E08C93089511
:102A100064FF03C081E08C9312C01C9210C02F573A
:102A2000304013963C932E93129783E08C9387E06B
:102A3000440F551F661F771F8A95D1F7706414964F
:102A40004D935D936D937C93179708951F93DC01CD
:102A5000FB019C91923008F447C08081823008F4D9
:102A600043C0943051F411961C91843099F58181C2
:102A7000682F70E0611B71093FC0843021F09230F3
:102A800031F48230B9F18181882389F12DC011960A
:102A90001C9111978230F1F081811817D9F41296A8
:102AA0002D913C911397828193818217930794F023
:102AB00028173907BCF014968D919D910D90BC910B
:102AC000A02D2481358146815781281739074A076F
:102AD0005B0718F4112341F00AC082179307A4077B
:102AE000B50740F4112319F061E070E005C06FEF05
:102AF0007FEF02C060E070E0CB011F910895991B49
:102B000079E004C0991F961708F0961B881F7A95E4
:102B1000C9F780950895AA1BBB1B51E107C0AA1FE6
:102B2000BB1FA617B70710F0A61BB70B881F991F6E
:102B30005A95A9F780959095BC01CD01089597FB12
:102B4000092E07260AD077FD04D0E5DF06D0002045
:102B50001AF4709561957F4F0895F6F790958195D9
:102B60009F4F0895A1E21A2EAA1BBB1BFD010DC0A9
:102B7000AA1FBB1FEE1FFF1FA217B307E407F5072D
:102B800020F0A21BB30BE40BF50B661F771F881F09
:102B9000991F1A9469F760957095809590959B019F
:102BA000AC01BD01CF0108952F923F924F925F92E9
:102BB0006F927F928F929F92AF92BF92CF92DF924D
:102BC000EF92FF920F931F93CF93DF93CDB7DEB7B2
:102BD000CA1BDB0B0FB6F894DEBF0FBECDBF099446
:102BE0002A88398848885F846E847D848C849B849D
:102BF000AA84B984C884DF80EE80FD800C811B81AB
:102C0000AA81B981CE0FD11D0FB6F894DEBF0FBED9
:0A2C1000CDBFED010895F894FFCF49
:102C1A004C697374206F66204D535220636F6D6D3B
:102C2A00616E64733A0A32392E30332E32303131C2
:102C3A000A45206F7220652020202020202D2D207B
:102C4A002020656E61626C65206368616E6E656CDA
:102C5A003A207479706520653F20666F722064653A
:102C6A007461696C65642068656C700A44206F72CF
:102C7A0020642020202020202D2D202064697361CB
:102C8A00626C65206368616E6E656C3A2074797057
:102C9A006520643F20666F722064657461696C65A3
:102CAA00642068656C700A6230206F72206231207D
:102CBA002020202D2D202073776974636820686591
:102CCA006172746265617420504134206F6E206FA6
:102CDA0072206F66660A47202020202020202020AC
:102CEA0020202D2D20202767657420414437373155
:102CFA003927202020202020202D3E206D65617359
:102D0A0075726520726573697374616E6365732089
:102D1A00616761696E0A6720202020202020202018
:102D2A0020202D2D2020276765742041546D65676A
:102D3A006120616463272020202D3E206D65617328
:102D4A0075726520766F6C74616765732020202028
:102D5A00616761696E0A50202020202020202020EF
:102D6A0020202D2D20206765742026207072696E20
:102D7A00742041443737313920696E66696E697447
:102D8A006C79200A7020202020202020202020205A
:102D9A002D2D20206765742026207072696E74209C
:102DAA0041546D6567612061646320696E66696E6E
:102DBA0069746C79200A732020202020202020208A
:102DCA0020202D2D20207072696E74207374617416
:102DDA0075730A48206F7220682020202020202D39
:102DEA002D20207072696E7420746869732068657A
:102DFA006C700A000A6572726F723A20696E7661A7
:102E0A006C69642027656E61626C6527206F722089
:102E1A002764697361626C652773746174656D6593
:102E2A006E742E0A0075736167653A205B457C658E
:102E3A007C447C645D5B727C767C687C705D5B3014
:102E4A002E2E31355D0A00652E672E3A20204576F2
:102E5A003120202D2D3E20656E61626C6520766FD3
:102E6A006C74616765206368616E6E656C20310AF7
:102E7A0000652E672E3A202064723020202D2D3EC8
:102E8A002064697361626C65207265736973746129
:102E9A006E6365206368616E6E656C20300A00613E
:102EAA006437373139206368616E6E656C733A2016
:102EBA00313520646F776E746F20303A0A0061648E
:102ECA0063206368616E6E656C7320313520646FB0
:102EDA00776E746F20303A0A20692E652E206C6551
:102EEA0066742069732070726573737572652061E8
:102EFA006E642068756D6964697479202E2E2E209F
:102F0A00726967687420697320766F6C746167658B
:102F1A000A000A20492077696C6C20737769746308
:102F2A006820006F6E20006F66662000207265734D
:102F3A00697374616E6365206368616E6E656C2087
:102F4A000020766F6C74616765206368616E6E65D8
:102F5A006C20002068756D69646974792063686102
:102F6A006E6E656C200020707265737375726520D1
:102F7A006368616E6E656C20000A2044414D4E21E3
:102F8A0020746869732073686F756C64206E657647
:102F9A0065722068617070656E2D20656E61626C65
:102FAA00652F64697361626C6520737769746368FD
:102FBA002D63617365210A000A686561727462652E
:102FCA00617420006F66660A006F6E0A0074696D8C
:102FDA00653A00207365632E0A000A6465627567A4
:102FEA00206D6F646520000A2072657369737461CD
:102FFA006E6365284F686D290A20286E6F74653ADA
:10300A00206F6E6C7920656E61626C6564206368FE
:10301A00616E6E656C7320617265207072696E7480
:10302A006564293A0A007C5200202020007C0A00AC
:10303A002020202020207C00566F6C746167652850
:10304A006D56292C202048756D6964697479286D3C
:10305A0056292020262020507265737375726528C0
:10306A006D56293A0A007C2056007C2048007C20B4
:10307A00500020202020202000567C00527C007224
:10308A0065636569766520627566666572206F7626
:10309A006572666C6F77202E2E2E207061727369AE
:1030AA006E67206E6F770A0050432073656E6469FD
:1030BA006E6720746F2066617374210A005839C8DC
:1030CA004001FA0177656C636F6D6520746F3A0A87
:1030DA00204D535220636F6D6D616E6420696E746A
:1030EA0065726661636520312E30200A2062756937
:1030FA006C643A2032392E30332E323031300A00A5
:10310A000304303132333435363738394142434497
:10311A004546000000000000000000000102020312
:10312A000303030404040404040404050505050553
:10313A000505050505050505050505060606060630
:10314A000606060606060606060606060606060615
:10315A000606060606060606060606070707070700
:10316A0007070707070707070707070707070707E5
:10317A0007070707070707070707070707070707D5
:10318A0007070707070707070707070707070707C5
:10319A0007070707070707070707070808080808B0
:1031AA000808080808080808080808080808080895
:1031BA000808080808080808080808080808080885
:1031CA000808080808080808080808080808080875
:1031DA000808080808080808080808080808080865
:1031EA000808080808080808080808080808080855
:1031FA000808080808080808080808080808080845
:10320A000808080808080808080808080808080834
:0C321A0008080808080808080808080050
:00000001FF
